:020000040800F2
:1000000000090020A1040008791300087D130008EE
:10001000B91300087D13000899130008A304000811
:10002000A3040008A3040008A30400081D35000869
:10003000A3040008A3040008A3040008A9390008C9
:10004000A3040008A3040008A3040008A3040008F4
:10005000A3040008A304000889370008B537000886
:10006000E13700080D38000839380008A3040008FB
:10007000A3040008A3040008A3040008A3040008C4
:10008000A3040008A3040008A3040008CD2400086A
:10009000392500088D250008E1250008653800088D
:1000A000A3040008A3040008A3040008A304000894
:1000B000A3040008A3040008A3040008A304000884
:1000C000A3040008A3040008A3040008A304000874
:1000D000A3040008052A0008192A0008A304000840
:1000E000CD380008A3040008A3040008A3040008F6
:1000F000A3040008A3040008A3040008A304000844
:10010000A3040008A3040008A3040008A304000833
:10011000A3040008A3040008A3040008A304000823
:10012000A3040008A3040008A3040008A304000813
:10013000A3040008A3040008A3040008A304000803
:10014000A3040008A3040008A3040008A3040008F3
:10015000A3040008A3040008A3040008A3040008E3
:10016000D0400B1CD1409C46203AD3401843524209
:1001700063469340184370479140031C90409C464F
:10018000203A9340194352426346D3401943704783
:1001900053B94AB9002908BF00281CBF4FF0FF31EE
:1001A0004FF0FF3000F07AB9ADF1080C6DE904CEE4
:1001B00000F006F8DDF804E0DDE9022304B0704742
:1001C0002DE9F0478C460E460446089D002B50D181
:1001D0008A4217466CD9B2FA82FEBEF1000F0BD0EC
:1001E000CEF1200C01FA0EF620FA0CFC02FA0EF702
:1001F0004CEA060C00FA0EF43A0CBCFBF2F9BBB266
:1002000002FB19CC09FB03FA4FEA144848EA0C46F2
:10021000B2450AD9F61909F1FF3180F02581B245BE
:1002200040F22281A9F102093E44A6EB0A06B6FB80
:10023000F2F002FB106600FB03F3A4B244EA0644AA
:10024000A34209D9E41900F1FF3280F00B81A342E7
:1002500040F2088102383C440021E41A40EA094097
:10026000002D62D0002324FA0EF42C606B60BDE8F0
:10027000F0878B4207D9002D55D0002185E8410039
:100280000846BDE8F087B3FA83F1002940F08F807B
:10029000B34202D3824200F2FC80841A66EB03066A
:1002A0000120B446002D40D085E81010BDE8F0874D
:1002B00012B90127B7FBF2F7B7FA87FEBEF1000FBC
:1002C00035D10121F61B4FEA174C1FFA87F8B6FB10
:1002D000FCF20CFB126608FB02F0230C43EA064614
:1002E000B04207D9F61902F1FF3302D2B04200F250
:1002F000D2801A46361AB6FBFCF00CFB106608FBDF
:1003000000F8A3B243EA0644A04507D9E41900F176
:10031000FF3302D2A04500F2B9801846A4EB0804CE
:1003200040EA02409CE729462846BDE8F08707FAE4
:100330000EF7CEF1200326FA03F24FEA174CB2FB78
:10034000FCF11FFA87F80CFB112206FA0EF620FAD0
:1003500003F301FB08F933431E0C46EA0246B1459C
:1003600000FA0EF409D9F61901F1FF3280F08C8001
:10037000B14540F2898002393E44A6EB0906B6FB3E
:10038000FCF00CFB106200FB08F99EB246EA024644
:10039000B14507D9F61900F1FF3371D2B1456FD9D4
:1003A00002383E44A6EB090640EA01418FE7C1F15D
:1003B000200722FA07F88B4048EA030326FA07F4DD
:1003C0004FEA134EB4FBFEF91FFA83FC0EFB1944EF
:1003D0008E4020FA07F809FB0CFA48EA06084FEAB3
:1003E000184646EA0444A24502FA01F200FA01F670
:1003F00008D9E41809F1FF3044D2A24542D9A9F145
:1004000002091C44A4EB0A04B4FBFEF00EFB1044EA
:1004100000FB0CFC1FFA88F848EA0444A44507D9FD
:10042000E41800F1FF3E29D2A44527D902381C4424
:1004300040EA0940A0FB0289A4EB0C0CCC45C24663
:10044000CE4615D312D055B1B6EB0A036CEB0E06AF
:1004500006FA07F7CB401F43CE402F606E600021A5
:10046000BDE8F0871046F7E68946DEE64645EAD263
:10047000B8EB020A69EB030E0138E4E77046D7E7F0
:1004800018468FE78146BDE7114676E702383C44BF
:1004900044E7084606E7023A3E442BE7704700BFB0
:1004A00002E000F000F8FEE772B6274880F3088803
:1004B000264880F3098826484EF60851CEF20001FE
:1004C0000860022080F31488BFF36F8F03F056F8A2
:1004D00003F0EEF84FF055301E491B4A91423CBFE5
:1004E00041F8040BFAE71C49184A91423CBF41F815
:1004F000040BFAE719491A4A1A4B9A423EBF51F8BF
:10050000040B42F8040BF8E700201749174A914200
:100510003CBF41F8040BFAE703F034F803F0CAF8E3
:10052000134C144DAC4203DA54F8041B8847F9E726
:1005300000F03AF8104C114DAC4203DA54F8041BA9
:100540008847F9E703F01CB80009002000110020DB
:10055000000000080001002000090020F040000811
:10056000001100207811002078110020D4250020EF
:1005700060010008600100086001000860010008D7
:100580002DE9F04FC1F80CD0C3689D46BDE8F08F4F
:10059000002383F311882846A047002002F0B4FD11
:1005A00002F05AFD00DFFEE76FF01702364B2DE92F
:1005B000F0411A70032200245A7001266FF0630282
:1005C0009C70DC701C715C719C71DC711C725A72C5
:1005D0009E72DC7202F04CFF804602F099FF0546E5
:1005E000D0BB2A4B984539D03344984537D0284B57
:1005F00028F0FF029A4234D15FFA88F000F04EFAF8
:100600002E4642F2107400F07FFC00F04DFA0746CF
:1006100058B364BB374635B11E4B984503D0002410
:1006200002F06EFF2746002002F02CFF1A4B9B6859
:1006300013F040031ED00FB100F030F800F086FC3C
:1006400000F020FE00F0C6FE0546ACB900F0D4FC78
:10065000012002F05FFDF8E70646D4E706462C4687
:10066000D1E706464FF47A74CDE70446D3E74FF45A
:100670007A74D0E71C46E1E700F0ACFE401BA042D4
:10068000E4D900F00BF8DDE778110020010007B095
:10069000000008B0263A09B0000C014010B51C4B10
:1006A0001C4953F8042F013200D110BD8B42F8D100
:1006B000194C1A4B22689A4228D9194B9B6803F1AE
:1006C000006303F5C8439A4220D202F0EDFE02F027
:1006D000FFFE002000F0F0FD0220124B187000F029
:1006E0001FFE114BDA690022DA61D96999699A61B2
:1006F0009B6972B60D4B0E4A202113601B6822685D
:1007000081F311889D4683F30888104710BD00BF10
:10071000FC6300081C64000804640008FF63000810
:1007200078110020841100200010024000640008AD
:1007300008ED00E049F2690008490B689AB21B0C09
:1007400000FB02330B6044F25061054A136898B213
:100750001B0C01FB0030106080B2704710110020AC
:100760000C11002010B504460021102200F0F4FD09
:10077000034B03CB206061601868A06010BD00BF10
:10078000E8F7FF1FF0B5BBB000F024FE1D4CA368D6
:10079000C31AF92B30D906AD2346A06028220021C8
:1007A000284601F0A5FB04F10E0000F0CDFD00236A
:1007B000C6B2591D5F1CDBB2B3424FEAC10107DA72
:1007C0000E3323440822284601F092FB3B46F0E713
:1007D00001230393082302930B4B207B01933023C7
:1007E000C1F3CF0105910093014604A3D3E900238F
:1007F0000495064801F04CF93BB0F0BD78F6339F04
:1008000093CACD8DC8210020D5210020A021002031
:1008100070B50D4614461E4601F0E0F850B9022EA0
:100820000ED1012C0CD112A3D3E90023C5E900237A
:10083000012070BD052C14D003D8012C09D0002054
:1008400070BD282C09D0302CF9D10BA3D3E900239B
:10085000ECE70BA3D3E90023E8E70BA3D3E90023DC
:10086000E4E70BA3D3E90023E0E700BFAFF3008088
:10087000401DA12026812A0B78F6339F93CACD8D87
:100880009E6AC421818A46EE26417272DF25D7B75F
:10089000F017304A39059E5638B50D4604460346D2
:1008A00020222846002101F023FB22792346032A37
:1008B00028BF0322284603F8042F2021022201F03A
:1008C00017FB62792346072A28BF0722284603F828
:1008D000052F2221032201F00BFBA2792346072AD0
:1008E00028BF0722284603F8062F2521032201F0FE
:1008F000FFFA284604F108031022282101F0F8FA33
:10090000382038BD2DE9F04FADF5037D23AE10AD95
:1009100040F2791280460F463046002100F01CFD5F
:1009200048220021284600F017FD00F053FD4FF447
:100930007A72B0FBF2F0574B0DF16209186093E840
:10094000070001232B74002385E807000DF16200E6
:100950006B74FFF707FF032385F82030E82385F841
:10096000213007AB18464C4903F088F8232228644D
:100970003146284685F83C20FFF78EFF14AB04462D
:1009800001460822304601F0B3FA08220DF1510366
:10099000A118304601F0ACFA0DF15203082204F11F
:1009A0001001304601F0A4FA15AB202204F1180121
:1009B000304601F09DFA16AB402204F13801304672
:1009C00001F096FA18AB082204F17801304601F0E4
:1009D0008FFA0DF16103082204F18001304601F025
:1009E00087FA04F1880A04F5847B4B4651460822B5
:1009F00030460AF1080A01F07BFAD34509F10109F2
:100A0000F3D11DAB08225946304601F071FA4FF080
:100A1000000904F5887495F834304B4510D84FF030
:100A2000000995F83C304B4515D92B6C21464B44B9
:100A30000822304601F05CFA083409F10109F0E7B8
:100A4000AB6B21464B440822304601F051FA083482
:100A500009F10109DFE7E31DC3F3CF03F97E059335
:100A6000002304960393BB7E193702930123019759
:100A70000093404605A3D3E9002301F009F80DF5E2
:100A8000037DBDE8F08F00BFAFF300809E6AC421F4
:100A9000818A46EE88110020343C0008014B187012
:100AA000704700BF94110020F0B52E4B85B01C7B21
:100AB0002CB10E222C4B1A81002005B0F0BD2B4A20
:100AC00002AB1068516803C3082329490DEB0302E8
:100AD000284802F0B5FF054630B90A22224B2648C5
:100AE0001A8100F041FCE7E70369B3F5CE3F07D96F
:100AF0000B211D4A21481181194600F035FCDBE726
:100B0000418BB1F57A7F08D00C22174B1C481A8113
:100B10004FF47A7200F028FCCEE71A4A103B0244E8
:100B2000144920469E1A00F059FC0746324605F14A
:100B30001801204600F052FCAB689F4202D1EB68DE
:100B400098420AD00D22084B1A8100903B46EA6871
:100B5000A9680D4800F008FCAEE70C4800F004FC62
:100B60000120AAE7C821002088110020243B0008AA
:100B7000DC9B0100006400082C3B0008383B0008A7
:100B80004A3B0008089CFFF7683B0008913B0008BF
:100B90002DE9F04FAFB006AF80460D4600F01EFFC6
:100BA000044600286CD12B7E022B18D1EB8A012B36
:100BB00015D100F00FFC8146FFF7BCFD4FF4C87360
:100BC000B0FBF3F202FB1300BD4E80B209F51679BB
:100BD000EB7E4844306093B90022BA4B1A70A437B8
:100BE000BD46BDE8F08F07F10C031C4400940023C0
:100BF00008224FEAC901284600F0DEFF4C46AB8AC6
:100C00005FFA84F9013BA3420BD904F10109B9F160
:100C1000110FE8D140F23911AB4BAC4AAC4802F0AD
:100C2000E1FE07F11C00FFF79DFD224607F11C01C4
:100C300007F10C0002F0F4FE03460028CCD1B9F114
:100C4000100F07D09F4B83F800903368A3F51673FD
:100C50003360C4E707F1A00202F8950D0146009247
:100C60002846072200F0A8FFF97A7F2904DD994B76
:100C7000964A4FF4A871D1E7404600F093FEAEE7E4
:100C8000EB8A052B00F02E8106D8012BA7D129462F
:100C90004046FFF737FEA2E7282B3DD0302B9ED1F0
:100CA0006B7E8D4C0133627BDBB29342EA4640F0AF
:100CB0000081EA7E237B9A4240F0FB80002607F108
:100CC000A00323F8846D00931022012331462846A7
:100CD00000F072FFB5F81480A8F102081FFA88F836
:100CE00008F1030323F003030A3323F00703ADEBFA
:100CF000030D0DF1180933469BB2B11C98454FEA1C
:100D0000C10106F101066DDD4B440093082200236A
:100D1000284600F051FFEEE7AB8A013B9BB2C92B9E
:100D20003FF65DAF6C4E347B4CBB06F10C03009379
:100D3000082223462146284600F03EFFAB8A04F1F4
:100D40000109013BE4B29C424FEAC90109DA0E34C1
:100D50003444009400230822284600F02DFF4C461E
:100D6000ECE700230022C6E900230023B36086F8E5
:100D7000D730C6F8D830337B0BB9EB7E3373002401
:100D800007F11C0607F10C03082221463046FC60DF
:100D90003C617C6101F0ACF83B7C04F10109A342A9
:100DA0004FEAC90107D97B6908222344304601F084
:100DB0009FF84C46F0E70023C1F3CF01E87E059190
:100DC00004960393AB7E19350293282301460093C2
:100DD000019539A3D3E90023404600F059FEFFF7FF
:100DE000D1FCFCE694F8D70000F078FAD4F8D830BB
:100DF00006461BB994F8D70000F080FAD4F8D83032
:100E000043449E4204D294F8D700013000F076FAB1
:100E10000025324B4FEA980BAAB25A45104616DA13
:100E20005AB994F8D72042B9D4E900120A4304D140
:100E3000D9F800201A600135EEE7226859F8201031
:100E400002EB80007B6000F039FA7B68F3E7D4E9BD
:100E50000023D4F8D85012EB080043F10001C4E994
:100E60000001454494F8D700C4F8D85000F036FA91
:100E7000854209D394F8D730013384F8D730D4F8B9
:100E8000D8309E1BC4F8D860B8F1FF0F0ADC0020F0
:100E9000124B2073196800F011FAFFF705FE08B134
:100EA000FFF7FCFB23680E4A9B0A013313810023E2
:100EB000A360D54693E600BF26417272DF25D7B7FF
:100EC0009C21002099210020A03B0008583C0008EC
:100ED000F93B00081B3C0008C8210020001100203D
:100EE00088110020BFF34F8F0549064BCA6802F4F2
:100EF000E0621343CB60BFF34F8F00BFFDE700BF3D
:100F000000ED00E00400FA0508B54FF000530B4A6D
:100F1000196891420AD1597D094A0A4811701B7D0E
:100F2000C922037308490E3000F004FABDE80840F6
:100F3000E02200214FF0005000F00EBA9AAD44C5F7
:100F400094110020C821002016000020022330B593
:100F50001F4C85B0637104230025ADF808300123D0
:100F60000722ADF80C501B498DF80C308DF80B3072
:100F7000194B1A484B608DF80A2001F0A9FD184B57
:100F8000019500931749184B4FF48052174800F011
:100F9000D3FC174B2546197811B1144800F002FD17
:100FA00000F018FA0446FFF7C5FB4FF4C873B0FB16
:100FB000F3F202FB130304F516749BB21C440D4BB1
:100FC0001C6002F0A5FA08B10F232B8105B030BDDB
:100FD000881100200411002003000600B822002020
:100FE0001108000898110020910B0008A021002092
:100FF000941100209C2100202DE9F04F96A7D7E9FD
:1010000000670FF25C29D9E900898F4C93B0DFF8B3
:1010100058B2DFF858A2204600F086FD0CAD0790CC
:1010200098B310220021284600F096F94FF00002F4
:10103000079B197B61F3030219468DF8302051F8A4
:10104000040F0EAA496803C21B680D9A584663F341
:101050001C029DF830300D9243F020038DF83030A3
:1010600000232A46194601F043FD079030B9204677
:1010700000F05EFD079B8AF80030CCE79AF800305C
:10108000072B40DC01338AF8003018220021284663
:1010900000F062F9DFF8D0B1DFF8D4A100232A46CE
:1010A0001946584601F04CFD014680BB102208A8A5
:1010B00000F052F9DAF80C3083F01003CAF80C3063
:1010C00000F08AF90DF1240E0B4612A9024611E92F
:1010D00003008EE803009DF83410C1F30300890675
:1010E00049BF0E99BDF83810C1F31C0141F0004111
:1010F00058BFC1F30A018DF82C000891204608A9B9
:1011000000F05CFFCAE7204600F012FDBDE7204674
:1011100000F064FC824600284AD100F05BF9DFF859
:1011200054B1DBF80030984242D300F053F90790F5
:10113000FFF700FB4FF4C873B0FBF3F101FB1300A2
:10114000079A80B202F516721044CBF80000DFF85F
:1011500028B18DF820A09BF8001011B901238DF85B
:10116000203028460791FFF7FDFA07990DF121007D
:10117000C1F1100A5FFA8AFABAF1060F28BF4FF0E0
:10118000060A2944524600F0D5F80AF101030493F7
:1011900008AB0393182302932C4B3246019301238F
:1011A000204600933B4600F01BFC00238BF80030E8
:1011B00000F010F9264ADFF8C4A01368C31AB3F58B
:1011C0007A7F32D3106000F007F902460B462046C2
:1011D00000F0B4FC204600F001FC30B39AF80C306B
:1011E000DFF89CB0002B14BF032302238BF80530DB
:1011F00000F0F0F84FF47A73B0FBF3F02946CBF827
:1012000000005846FFF748FB18230293114B0730A4
:10121000019340F25513C0F3CF000490009303955F
:1012200042464B46204600F0DBFB9AF80C300BB1EF
:10123000FFF7A8FA9AF80C30002B7FF4E8AE13B051
:10124000BDE8F08FAFF30080A0210020982100209E
:10125000A8220020AC220020401DA12026812A0BBC
:10126000F1C6A7C1D068080FB8220020AD22002027
:10127000000801409C21002099210020C821002065
:101280008811002070B501F0FBFF0025084C094EC5
:10129000207030682378834208D901F0EDFF33686D
:1012A00005440133B5F5C84F3360F2D370BD00BFBC
:1012B000B4220020B022002002F070B807B502ABC3
:1012C00043F8041D00F100600422194600F5C840EF
:1012D00002F010F803B05DF804FB0000054B1A683B
:1012E000054B1B789B1A834202D9104401F0C4BFFE
:1012F00000207047B0220020B422002038B50446F8
:10130000064D2868204401F0BDFF28B92868204414
:10131000BDE8384001F0C8BF38BD00BFB022002092
:10132000022802BF4FF48012014B1A61704700BFC0
:1013300000080140002310B5934203D0CC5CC45494
:101340000133F9E710BD000002460346981A13F96D
:10135000011B0029FAD1704703460244934202D090
:1013600003F8011BFAE770470FB4002004B0704780
:101370000EB4002003B07047FEE70000EFF30983CE
:10138000EFF30583034B9A6B9A6A9A6A9A6A9A6A90
:101390009B6AFEE700ED00E0EFF30983EFF30583BE
:1013A000044B9A6B9A6A9A6A9A6A9A6A9A6A9B6AD0
:1013B000FEE700BF00ED00E0EFF30983EFF30583E4
:1013C000034B5A6B9A6A9A6A9A6A9A6A9B6AFEE710
:1013D00000ED00E002F01AB801F0F4BF30B5084D9E
:1013E0000A4491420BD0092411F8013B5840013CBA
:1013F000F7D040F300032B4083EA5000F7E730BDFD
:101400002083B8ED0246006848B103681189136073
:10141000D38801339BB29942D38038BF1381704780
:1014200070B504460D4688B0202200216846FFF7BB
:1014300093FF20460495FFF7E5FF054658B16B463C
:10144000044608AE1A4603CAB242206061601346E1
:1014500004F10804F6D1284608B070BD2DE9F0412A
:1014600030B940F2C531264B264A274802F0BAFA75
:101470000B7C23B9254B234A40F2C631F5E7C669F8
:1014800086B9C161BDE8F081002B29DA930CAB422B
:1014900029D1B44201D10C60F3E7C8F800100C6008
:1014A000BDE8F0814B68B04623F06047BD0C15EAFB
:1014B000230538BF3D4634464FEAD37EC3F3807CD4
:1014C0006368BEEBD37F23F06042DDD1974203D146
:1014D000C3F380739C450AD1974205E01C46EFE7B1
:1014E000AA4206D013469D422CBF00230123002BA5
:1014F000CFD12368A046002BF0D12160BDE8F08158
:101500002C3F0008203D0008E43F0008054000088B
:1015100008B5034A034B40F25E31034802F062FA19
:10152000FC3C0008A43F0008E43F000808B503683D
:101530000B60C388016033B9044B054A4FF4C7619F
:10154000044802F04FFA013BC38008BD743F000815
:10155000703D0008E43F000870B50C4600F10C0532
:10156000616831B9E38A002061F30903E382002155
:1015700070BD0E682846FFF7D9FF6660F0E70000EF
:1015800008B5426832B10B4B0B4A40F22F410B4871
:1015900002F028FAC37DC3F38401013161F38603AD
:1015A000C375C38A62F30903C3821B0A62F3C713BC
:1015B000C37508BDC03F00082C3D0008E43F00088B
:1015C0002DE9F047089E32B91F4B204A40F23951AD
:1015D0001F4802F007FA4FF47F4901F007054FEA70
:1015E000D6082A4406F0070600EBD100954201D147
:1015F000BDE8F08705F0070E06F0070AD6457746E6
:1016000038BF5746511BC7F108078F4228BF0F4606
:10161000EC08045D08EBD60113F801C004FA0EF4DF
:1016200029FA07FE24FA0AF45FFA8EFE8CEA040413
:101630004EFA0AFE04EA0E048CEA040C03F801C018
:101640003D443E44D2E700BF403F0008443D00080F
:10165000E43F00082DE9F04106460F4600254FF60D
:10166000FF7441F221082A4630463946FEF778FDDC
:101670000823C0B284EA002414F4004F4FEA440463
:10168000A4B203F1FF3318BF84EA080413F0FF0388
:10169000F2D10835402DE6D12046BDE8F0810000AA
:1016A00010B541F221040A44914200D110BD11F855
:1016B000013B80EA0320082310F4004F4FEA40006A
:1016C00080B203F1FF3318BF604013F0FF03F3D182
:1016D000EAE700002DE9F04F85B08A468DE80C005E
:1016E000BDF83C40814630B940F26E31484B494A22
:1016F000494802F077F911F0604F04D0474B454A52
:1017000040F26F31F4E7009B002B7ED024B10E9B9A
:10171000002B7AD0072C28D809F10C00FFF772FEB5
:10172000054628B96FF00205284605B0BDE8F08FE0
:1017300014220021FFF710FE22460E9905F1080041
:10174000FFF7F8FD631C2B74009B2C441B78294683
:1017500003F01F0363F03F0323724AF000436B6002
:101760004846FFF77BFE0125DEE74FF000084FF00B
:10177000800B46464546019B1B0A029300F10C0371
:1017800003930398FFF73EFE07460028CAD01422B1
:101790000021FFF7E1FDB6BB02229DF804303B7249
:1017A0009DF808307B720E9B711E1944B4420AD911
:1017B000B818013211F801EFD2B20136072A80F8C9
:1017C00008E0B6B2F2D1B44208BF4FF0400B009B24
:1017D000B8181978013201F01F0141EA48114BEAAB
:1017E000010303724AF000437B603A74394648466D
:1017F000FFF734FE0135B4422DB288F001084FF0F6
:10180000000BBED190E70022CDE76FF001058BE71A
:101810002C3F0008103D0008E43F0008503F00083E
:101820002DE9F0471E46CB8A9146C3F30902062AEA
:1018300080460F4619D013460021B0B28DB25A1916
:1018400092B2052A09D9A84210D8FA8A034463F350
:101850000902FA820120BDE8F087A842F3D919F8FD
:1018600001403A4494760131E8E70025FB8A7C6820
:10187000C3F309001C23821FB2FBF3FA03FB1A2AED
:101880001FFA8AF27CB301212368002B39D1B31FE0
:1018900003441C20B3FBF0F301339BB299420CD2FA
:1018A000BAF1000F09D14046FFF7ACFD08B1C0F80E
:1018B00000A0206008B3044600224FF0000AB6B230
:1018C000B54230D21346691E4944E018013311F87D
:1018D00001EF9BB201351C2B80F804E0ADB214D0AF
:1018E000AE42F2D8ECE74046FFF78CFD044608B163
:1018F000002303607C60002CDED16FF00200BDE8A5
:10190000F087013189B21C46BEE7AE42D8D94046C5
:10191000FFF778FD08B1C0F800A020600028ECD0E7
:1019200004460022CCE7FB8AC3F30902164466F39F
:101930000903FB828EE70000F8B50E4615461F46E8
:10194000044628B9144B154A4F21154802F04AF8AD
:1019500024220021FFF700FD069B6A096360079BB4
:10196000002023624FF6FF739A4228BF1A46A760F1
:101970002070A061E06197B204F10C05824205D1AC
:1019800000232B6027826382A382F8BD2E60013082
:1019900035462036F2E700BF283F00089C3C00088F
:1019A000E43F000808B528B97321084B084A0948E4
:1019B00002F018F8037823B94BB2002B01DD017057
:1019C00008BD054B024A7D21F1E700BF2C3F00080E
:1019D000A83C0008E43F0008703E0008007870470B
:1019E0002DE9F7430D9E074619461046BDF828908D
:1019F0000B9D9DF83040BDF8388016B9B8F1000F46
:101A000043D11F2C41D83B78D3B9B8F1070F39D84F
:101A100039F0030339D1424631464FF6FF70FFF7E4
:101A20003FFE4FEA092920F0010009F44079400403
:101A300049EA0464400C44EA40244FF6FF730DE089
:101A400043EA0923B8F1070F43EA0464F5D9FFF725
:101A500001FE42463146FFF723FE03468DE8400172
:101A60002A4621463846FFF735FE0DB9FFF750FDEF
:101A70002B780133DBB21F2B88BF00232B7003B000
:101A8000BDE8F0836FF00300F9E76FF00100F6E7BF
:101A90002DE9F7430E9F81460B9D9DF830009DF880
:101AA0003480BDF83C6007B9C6BB1F2836D899F80A
:101AB00000E0BEF1000F34D00C0244F080049DF829
:101AC000281044EAC83444EA014444EA0E04072ECC
:101AD00044EA006415D919461046FFF7BBFD3246AB
:101AE0003946FFF7DDFD0346019600972A46214659
:101AF0004846FFF7EFFDB8F1010F0CD125B9FFF70C
:101B000007FD4FF6FF73EFE72B780133DBB21F2B96
:101B100088BF00232B7003B0BDE8F0836FF0010095
:101B2000F9E76FF00300F6E7C06900B104307047D1
:101B3000C1690C300B680361FFF7F8BC2DE9F84F61
:101B4000D0F818A0054616461F4654464FF0000927
:101B5000DFF8608000F10C0B0CB9BDE8F88FD4E918
:101B60000223B21A67EB0303994508BF90451FD2C1
:101B7000AB6921469C4228460DD1FFF7EDFCAB69CD
:101B800021461B685846AB61FFF7D0FCAC69234681
:101B9000A2461C46E0E7FFF7DFFC23682146CAF8AF
:101BA00000305846FFF7C2FC5446DAF80030EFE741
:101BB0002368EDE780841E002DE9F04F8BB00D46C1
:101BC00014460793DDF850908246002800F06481A7
:101BD000B9F1000F00F06081531E3F2B00F25C81D1
:101BE000012A03D1079B002B40F056810023BAF84D
:101BF00014600893F600B542099380F053812B19C5
:101C00009E420AD2761B16F0FF0607D140F26751BA
:101C1000AA4BAB4AAB4801F0E5FE2646DAF80C3099
:101C200023B9DAF81030002B00F0A5802F2D31D821
:101C3000C5F1300846454FF0000334BFB0465FFAA7
:101C400088F80093294608AB4246DAF80800FFF707
:101C5000B7FCA6EB08074544FFB24FF0300BBAF8CB
:101C6000143003F10053063BDB000293DAF80C302A
:101C70000593059B002B51D087B9DAF81000002896
:101C800061D0002F5FD0AB4550D98F4B8C4A40F2CA
:101C9000A651BFE737464FF00008DEE7029B23B9A5
:101CA0008A4B874A4FF4B161B4E7029BE02B28BF0F
:101CB000E02306935B44AB4204931DD95B1B9F4218
:101CC00026BFDBB203930397AB4504D97E4B7C4A16
:101CD00040F291519EE70598CDF8008008ABA5EB46
:101CE0000B01039A0430FFF76BFC039B9844FF1A27
:101CF0001D445FFA88F8FFB2049B9B4504D3744BE4
:101D00006F4A40F29B5185E7029B069ADDF810B0BE
:101D10009B1A0293059B1B680593AAE7029BBB4293
:101D2000ABD26C4B664A40F2A15173E7CDF800800C
:101D30003A46A5EB0B0108ABB8443D44FFF740FC25
:101D400000275FFA88F8BAF81430B5EBC30F04D94E
:101D5000614B5B4A40F2B1515CE7B8F1400F04D9E6
:101D60005E4B574A40F2B25154E767B15C4B544A5C
:101D700040F2B3514EE70093324608AB2946DAF8F9
:101D80000800FFF71DFC731E3F2B35B201D8A64299
:101D900004DD544B544A40F235213BE760070AD03A
:101DA0000AAB03EBD40111F8083C624202F00702CF
:101DB000134101F8083C082C21D9102C21D9202CE2
:101DC0008CBF08230423079A002A6DD0B4EBC30FFD
:101DD0006CD0082C04F1FF3215D89DF8203023FA7E
:101DE00002F2D10706D54FF0FF3202FA04F4234382
:101DF0008DF820309DF8203089F800304EE0012326
:101E0000E1E70223DFE7102C11D8BDF8203023FAD8
:101E100002F2D20706D54FF0FF3202FA04F4234350
:101E2000ADF82030BDF82030A9F8003036E0202C85
:101E30000ED8089921FA02F2D30705D54FF0FF33E7
:101E400003FA04F40C430894089BC9F8003025E019
:101E5000402C1CD0DDE9086730463946FEF780F992
:101E6000002100F0010050EA01030BD022460120BE
:101E70000021FEF781F9404261EB410106430F4327
:101E8000CDE90867DDE90823C9E9002306E0174B1F
:101E9000154A4FF42071BDE66FF0010528460BB0DE
:101EA000BDE8F08F1D46F9E7012CA3D0082CA1D97D
:101EB000102CB7D9202CE5D8C6E700BF7C3D000820
:101EC000543D0008E43F00089E3D00088B3D00089B
:101ED000C33D0008EB3D0008123E0008403E0008EC
:101EE000583E0008723E0008D43C0008703E0008CE
:101EF00030B585B030B940F2B121234B234A244894
:101F000001F070FD23B9234B204A40F2B221F6E7DD
:101F1000402A04D9204B1D4A40F2B621EFE722B9EE
:101F20001D4B1A4A4FF42F71E9E70024012A02944D
:101F3000039417D11B788DF8083053070AD004ABEF
:101F400003EBD20313F8084C554205F00705AC40EB
:101F500003F8084C00910346002102A8FFF730FB6C
:101F600005B030BD082AE5D9102A03D81B88ADF882
:101F70000830E2E7202A02D81B680293DDE7D3E9A4
:101F80000045CDE90245D8E7AC3E0008E83C000832
:101F9000E43F0008C73E0008703E000870B50C46DC
:101FA00000F10C05E16819B9A1602161A18270BD41
:101FB0000E682846FFF7BAFAE660F3E72DE9F04F1E
:101FC000D1F8009091B0C9F3C01604460D46CDE992
:101FD0000223002E50D0C9F3C03BC9F30626B9F145
:101FE000000F80F29F8119F0C04F40F09B812B7B46
:101FF000002B00F09781BBF1020F03D02278B24290
:1020000040F0938109F07F02BBF1020F059236D1B7
:1020100019F07F0FC9F30F2A01D10AF0030A2B44EC
:102020007606059A93F8038046EA0B4646EA82460E
:102030005FEAD81346EA0A06069300F09A80002267
:10204000002310A961E90823059B676800935246A5
:102050005B462046B847002800F08880A7698FB902
:10206000314604F10C00FFF7DBF90746D0B96FF0F9
:10207000020011B0BDE8F08F4FF0020BAFE7C9F3DB
:10208000074ACCE73B699E420DD03F68002FF9D14B
:10209000314604F10C00FFF7C3F907460028E6D0EB
:1020A000A3693B60A761DDE90801FFF7D3FAB882B5
:1020B000F97D08F01F06C1F38401711A89B20FFA85
:1020C00081FEBEF1000FB8BF01F1200EC9F304611B
:1020D000D7E90223B8BF0FFA8EFE079152EA030137
:1020E00000F02F81DDE90201801A61EB03010B464C
:1020F000002102469E48994208BF9042C0F02181CB
:10210000069B002B3FD0BEF1010F00F31A8118F09F
:10211000400F38D0DDE90223C7E902232022002145
:102120000DEB0200FFF718F9DDE90223CDE90823E2
:102130002B1D0A932B7B2046013BDBB2ADF83430DC
:102140009DF81C30ADF836A08DF83A309DF814306B
:102150008DF838B08DF83B308DF83960A36808A948
:1021600098473846FFF70CFA002082E76FF00B0023
:102170007FE7A76917B96FF00C007AE73B699E42C9
:1021800096D03F68F6E7FB7DC8F34012B2EBD31F51
:1021900040F0CE80C3F38403B34240F0CC80069974
:1021A0002B7B4FEA981279B3D2073CD4032B40F231
:1021B000C580DDE90223C7E902232B7BAE1D033B6B
:1021C000DBB23246394604F10C00FFF729FB002848
:1021D00008DA39462046FFF7BFF93846FFF7D0F94D
:1021E000032046E7AB883B832A7B033AD2B2B88A06
:1021F0003146FFF755FAFB7DB882DA43C2F3C012CD
:1022000062F3C713FB75AFE76AB92E1D013BDBB262
:102210003246394604F10C00FFF702FB0028D8DBF8
:102220002A7B013AE2E7FA8A013BC2F30902052A56
:10223000D9B250D80023281D99420AD907EB020EC3
:1022400010F801CB01320133062A8EF81AC0DBB236
:10225000F2D18B4228BF0023DDE9028907F11A027F
:10226000CDE908890A927A683CBF04335B190B9266
:102270000C93FB8AADF836A0C3F3090319449DF80B
:102280001C30ADF834108DF83A309DF814308DF8CC
:1022900038B08DF83B3000238DF839607B602A7BA5
:1022A000B88A013A291DFFF7FBF93B8BB8828342BC
:1022B00003D1A36808A92046984708A92046FFF73C
:1022C0006DFE3846FFF75CF9B88A3B8B984214BF25
:1022D00011200020CDE6786810B34FF0060E036899
:1022E0009BB9A2EB0E021B2A13D80332024405F15C
:1022F000040E1F309942ACD91EF801CB013302F80D
:1023000001CF9042DBB2F5D1A3E70EF11C0E1846C7
:10231000E5E7184B184A40F2B311184801F062FB88
:10232000034696E76FF00900A3E66FF00A00A0E607
:102330006FF00D009DE66FF00E009AE66FF00F0053
:1023400097E6FB7D394668F386036FF3C713FB7589
:102350002046FFF701F9069B002B7FF4D8AEFB7DEA
:10236000C3F38402013262F38603FB7503E700BF07
:1023700080841E00DC3E0008C03C0008E43F0008EA
:102380002DE9F0414E4EB04240F086804D4CDFF8D2
:1023900038E1E56945F00075E561E469846AD4F8DF
:1023A000007207EA0E0747F00107C4F80072D4F87C
:1023B000005205EA0E0545F0010545EA0121C4F881
:1023C0000012002A6AD000210F46C4F81C12C4F87B
:1023D0000412C4F80C12C4F8141204EBC105013144
:1023E0000E29C5F84072C5F84472F6D14FF0000EC0
:1023F0004FF0010C964510D1826AB042D2F80032FB
:1024000023F00103C2F8003258D12E4BDA6922F0D2
:102410000072DA61DB69BDE8F0819F781D8817F0F2
:10242000010F18BFD4F804820CFA05F11CBF41EA71
:102430000808C4F8048217F0020F18BFD4F80C8201
:1024400004EBC5051CBF41EA0808C4F80C827F07ED
:1024500048BFD4F8147203F10C0344BF0F43C4F80F
:10246000147253F8087C0EF1010EC5F8407253F84F
:10247000047CC5F84472D4F81C522943C4F81C12D9
:10248000B8E70021846AC4F81C12C4F80412C4F826
:102490000C12C4F81412A9E7002AF2D10022836AB0
:1024A000C3F84022C3F84422C3F80422C3F814221C
:1024B0000122C3F80C22C3F81C229DE7BDE8F0817D
:1024C000B8220020001002400000FFFF184A08B5A3
:1024D000916A8B688B6013F0010105D013F00C0F2B
:1024E00014BF4FF480310121D80506D513F4406F95
:1024F00014BF41F4003141F00201D80306D513F4B2
:10250000402F14BF41F4802141F00401D3690BB185
:1025100007489847202383F311880021054800F0DD
:1025200021FE002383F31188BDE8084001F000B8C4
:10253000B8220020C022002038B5124CA36ADD6802
:10254000AA0712D05A6922F002025A61A36913B194
:10255000012120469847202383F3118800210A484F
:1025600000F000FE002383F31188EB0606D510214E
:10257000A36AD960236A0BB102489847BDE8384086
:1025800000F0D6BFB8220020C822002038B5124C77
:10259000A36A1D69AA0712D05A6922F010025A6173
:1025A000A36913B1022120469847202383F31188A1
:1025B00000210A4800F0D6FD002383F31188EB06C2
:1025C00006D51021A36A1961236A0BB10248984706
:1025D000BDE8384000F0ACBFB8220020C82200207F
:1025E00038B50F4CA36A5D682A075D600AD50322DF
:1025F00022701A6822F002021A60636A13B1002185
:10260000204698476B0706D5A36A9969236A13B1D8
:10261000090403489847BDE8384000F089BF00BF6F
:10262000B822002010B50F4C204600F03FFA0E4BA8
:102630000B211320A36200F019FA0B21142000F0E3
:1026400015FA0B21152000F011FA0B21162000F0CD
:102650000DFA00232046BDE810401A460E21FFF770
:102660008FBE00BFB8220020006400400F4B10B5A1
:102670009842044605D10E4BDA6942F00072DA61E5
:10268000DB690122A36A1A60A36A5A68D20707D5D8
:10269000626851681268D9611A60064A5A6110BDB1
:1026A0000121082000F092FCEEE700BFB8220020D4
:1026B000001002405B87010003291AD8DFE801F00F
:1026C000020A0F14836A9B6813F0E05F14BF0120B5
:1026D00000207047836A9868C0F380607047836AFF
:1026E0009868C0F3C0607047836A9868C0F3007050
:1026F000704700207047000010B503291FD8DFE89D
:1027000001F0021F2327816A8B68C3F3016318332A
:1027100001EB0313107881061ED55468C0F3001135
:10272000490041EAC40141F0040100F00F00586083
:10273000906841F001019860D268DA60196010BDBC
:10274000836A03F5C073E5E7836A03F5C873E1E7BD
:10275000836A03F5D073DDE79488C0F30011490064
:1027600041EA4451E1E7000001290CD003D30229DA
:1027700010D000207047836ADA68920701D1186987
:1027800003E001207047836AD86810F0030018BF87
:1027900001207047836AF2E710B539B9836AD968B6
:1027A00089071BD11B699B0704D110BD012915D0D6
:1027B000022948D1816AD1F8C031D1F8C401D1F8D9
:1027C000C8411461D1F8CC41546120240C610C69DA
:1027D000A40717D14C6944F0100412E0816AD1F8C3
:1027E000B031D1F8B401D1F8B8411461D1F8BC418D
:1027F00054612024CC60CC68A40703D14C6944F018
:1028000002044C6111795C0864F304119C0864F3C0
:102810004511117189064BBF91681189DB085B0D69
:102820004CBF63F31C0163F30A01137948BF916045
:1028300060F3030313714FEA10234FEA104058BFAF
:1028400011811370508010BD00231A4610B51C4929
:102850005A50CC180833802B6260F9D1194B9A6911
:1028600042F07D029A619B690268174BDA608268C8
:102870005A6042681A60C26803F58063DA60426990
:102880005A6002691A608269C3F80C24026AC3F8AC
:102890000424C269C3F80024426AC3F80C28C26A3F
:1028A000C3F80428826AC3F80028026BC3F80C2C12
:1028B000826BC3F8042C426BC3F8002C10BD00BF20
:1028C000E422002000100240000801400268436832
:1028D0001143016003B1184770470000024AD368F2
:1028E00043F0C003D360704700380140024AD36808
:1028F00043F0C003D3607047004400402DE9F0412D
:10290000D0F89C600546F7683368DA059CB20DD5AF
:10291000202383F311884FF400710430FFF7D6FFB2
:102920006FF480733360002383F31188202383F3D3
:10293000118805F1040814F02F0333D183F31188B3
:10294000380615D5210613D5202383F3118805F108
:10295000380000F02FFA002846DA0821281DFFF77A
:10296000B5FF4FF67F733B40F360002383F311887C
:102970007A060ED563060CD5202383F31188EA6C02
:102980002B6D9A4202D12B6C002B2FD1002383F3A5
:102990001188D5F8A420D368002B31D0BDE8F041D0
:1029A00010691847230713D014F0080F0CBF00213B
:1029B0008021E00748BF41F02001A20748BF41F055
:1029C0004001630748BF41F480714046FFF77EFF36
:1029D000A406736805D595F8A0102846194000F0A4
:1029E00089FA3468A4B2A6E77060BEE727F0400712
:1029F0003F041021281D3F0CFFF768FFF760C5E773
:102A0000BDE8F08108B50348FFF778FFBDE808404E
:102A100000F08EBD6423002008B50348FFF76EFF69
:102A2000BDE8084000F084BD0C24002010B5094C1E
:102A3000094A2046002100F03DFA084B084AC4F834
:102A40009C30084C0021204600F034FA064BC4F8B4
:102A50009C3010BD64230020DD28000800380140B0
:102A6000ED2800080C2400200044004000F16043E1
:102A7000090103F56143C9B283F80013012300F093
:102A80001F024009800000F16040934000F5614062
:102A9000C0F8803103607047090100F16040C9B29D
:102AA00000F56D4001767047FFF7BCBD0123037050
:102AB000002300F108028260C26000F1100243604E
:102AC000026142618361C361036243627047000037
:102AD00010B52023044683F311880223416003705C
:102AE000FFF7C4FD03232370002383F3118810BD77
:102AF0002DE9F0411F4604460D461646202383F378
:102B0000118800F108082378042B0ED029462046AE
:102B1000FFF7D2FD48B1204632462946FFF7ECFDCB
:102B2000002080F31188BDE8F0813946404600F06E
:102B3000FDFA0028E7D0002383F31188BDE8F08177
:102B40002DE9F0411F4604460D461646202383F327
:102B5000118800F110082378042B0ED02946204656
:102B6000FFF702FE48B1204632462946FFF714FE21
:102B7000002080F31188BDE8F0813946404600F01E
:102B8000D5FA0028E7D0002383F31188BDE8F0814F
:102B9000F8B5154682680B46AA428169066938BFB6
:102BA0008568761AB542044607D218462A46FEF7CB
:102BB000C1FBA3692B44A3610DE011D9324618462D
:102BC000FEF7B8FBAF1B3A46E1683044FEF7B2FBB4
:102BD000E2683A44A261A36828465B1BA360F8BD83
:102BE00018462A46FEF7A6FBE368E4E72DE9F04124
:102BF0000446154683682669934238BF8568406954
:102C00000F46361AB54206D22A46FEF793FB636991
:102C10002B4463610DE012D93246A5EB0608FEF79E
:102C200089FB4246B919E068FEF784FBE26842443A
:102C30006261A36828465B1BA360BDE8F0812A4659
:102C4000FEF778FBE368E4E710B50024C361029B5C
:102C50000A44006040608460C1608161416102613A
:102C6000036210BD08B582694369934201D182684D
:102C700082B98268013282605A1C426119704269CD
:102C800003699A4201D3C3684361002100F05EFAF0
:102C9000002008BD4FF0FF3008BD000070B52023B4
:102CA00004460E4683F31188A568A5B1A368A269FE
:102CB000013BA360531CA36115782269934224BF92
:102CC000E368A361E3690BB120469847002383F3CF
:102CD0001188284670BD3146204600F027FA0028AA
:102CE000E2DA85F3118870BD2DE9F74F05460F46EE
:102CF00090469A46D0F81C90202686F311884FF013
:102D0000000B144664B1224639462846FFF740FFBF
:102D1000034668B95146284600F008FA0028F1D069
:102D2000002383F31188A8EB040003B0BDE8F08F03
:102D3000B9F1000F03D001902846C847019B8BF3DF
:102D40001188E41A1F4486F31188DBE7C361009BF6
:102D5000C160816141611144006040608260016135
:102D600003627047F8B504460E461746202383F3E6
:102D70001188A568A5B1A368013BA36063695A1CCB
:102D800062611E70236962699A4224BFE3686361CD
:102D9000E3690BB120469847002080F31188F8BD05
:102DA0003946204600F0C2F90028E2DA85F311889E
:102DB000F8BD00008369426910B59A4201D182686A
:102DC0007AB98268013282605A1C82611C78036978
:102DD0009A4201D3C3688361002100F0B7F920460D
:102DE00010BD4FF0FF3010BD2DE9F74F05460F46DF
:102DF00090469A46D0F81C90202686F311884FF012
:102E0000000B144664B1224639462846FFF7EEFE11
:102E1000034668B95146284600F088F90028F1D0E9
:102E2000002383F31188A8EB040003B0BDE8F08F02
:102E3000B9F1000F03D001902846C847019B8BF3DE
:102E40001188E41A1F4486F31188DBE7026843689F
:102E50001143016003B11847704700001430FFF7B9
:102E600043BF00004FF0FF331430FFF73DBF0000B9
:102E70003830FFF7B9BF00004FF0FF333830FFF7AD
:102E8000B3BF00001430FFF709BF00004FF0FF315F
:102E90001430FFF703BF00003830FFF763BF0000B6
:102EA0004FF0FF323830FFF75DBF00000020704761
:102EB000FFF7BCBD0E4B37B5036000234360836052
:102EC000C3600123044615460374202200900B467C
:102ED00000F15C011430FFF7B7FE00942B4620226E
:102EE00004F17C0104F13800FFF730FF03B030BD7E
:102EF0002040000838B5C36904460D461BB90421BB
:102F00000844FFF7A3FF294604F11400FFF7AAFEC7
:102F1000002806DA201D4FF48061BDE83840FFF735
:102F200095BF38BD0022024B1B605B609A60704702
:102F3000B4240020002382680374054B1B68996841
:102F40009142FBD25A68036042601060586070473B
:102F5000B424002008B5202383F31188037C032BBD
:102F600005D0042B0DD02BB983F3118808BD0022A6
:102F700043691A604FF0FF334361FFF7DBFF002323
:102F8000F2E790E80C001A6002685360F2E7000074
:102F9000002382680374054B1B6899689142FBD833
:102FA0005A6803604260106058607047B424002083
:102FB000054B196908741868026853601A60186133
:102FC00001230374FDF7DCBAB424002030B54B1C98
:102FD00087B005460A4C10D023690A4A01A800F0C0
:102FE000DDF82846FFF7E4FF049B13B101A800F0C9
:102FF000EFF82369586907B030BDFFF7D9FFF8E74C
:10300000B4240020552F000838B50C4D41612B69C0
:1030100081689A680446914203D8BDE83840FFF7BA
:1030200089BF1846FFF786FF01232C6101462374F0
:103030002046BDE83840FDF7A3BA00BFB424002005
:10304000044B1A681B6990689B68984294BF0020E3
:1030500001207047B424002010B5084C2368206973
:103060001A6854602260012223611A74FFF790FFEE
:1030700001462069BDE81040FDF782BAB424002063
:1030800008B5FFF7DDFF18B1BDE80840FFF7E4BF62
:1030900008BD000082600222027400224274704760
:1030A0008368A3F13C0243F80C2C026943F83C2CE2
:1030B000426943F8382C074A43F81C2CC268A3F134
:1030C000180043F8102C022203F8082C002203F801
:1030D000072C70479105000810B5202383F3118851
:1030E000FFF7DEFF00210446FFF78EFF002383F386
:1030F0001188204610BD0000024B1B6958610F204B
:10310000FFF756BFB4240020202383F31188FFF774
:10311000F3BF000008B50146202383F3118808207F
:10312000FFF754FF002383F3118808BD49B1064B14
:1031300042681B6918605A60136043600420FFF7FF
:1031400045BF4FF0FF307047B42400200368984219
:1031500006D01A680260506059611846FFF7EABE4F
:103160007047000038B504460D462068844200D1FF
:1031700038BD036823605C604561FFF7DBFEF4E760
:10318000054B03F114025A619A614FF0FF32DA6184
:1031900000221A62704700BFB424002010B5C2603C
:1031A0000A4A036153699C68A1420CD85C680360B9
:1031B00044602060586081609868411A99604FF0BF
:1031C000FF33D36110BD091B1B68ECE7B42400205A
:1031D000036881689A680A449A60426813600368C9
:1031E0005A6000234FF0FF32C360014BDA61704731
:1031F000B424002000207047FEE700007047000064
:103200004FF0FF3070470000BFF34F8F024AD36882
:10321000DB07FCD4704700BF0020024008B5074B15
:103220001B7853B9FFF7F0FF054B1A69120641BF2F
:10323000044A5A6002F188325A6008BD0425002011
:10324000002002402301674508B5054B1B7833B9C0
:10325000FFF7DAFF034A136943F08003136108BDE7
:1032600004250020002002407F289ABF00F500308E
:1032700080020020704700004FF48060704700001B
:10328000802070477F2808B50BD8FFF7EDFF00F5C9
:1032900080630268013204D104308342F9D10120F5
:1032A00008BD002008BD00007F2810B504461CD8CA
:1032B000FFF7AAFFFFF7B2FFF3220D4BDA600222FD
:1032C0001A61FFF7D1FF58611A6942F040021A6192
:1032D000FFF79AFF4FF4806100F0E4F8FFF7B4FFC6
:1032E0002046BDE81040FFF7CDBF002010BD00BF55
:1032F000002002402DE9F84312F00103144606D0E5
:1033000040F241221F4B1A600020BDE8F883851867
:103310001D4A954204D940F246211A4A1160F3E74A
:10332000FFF77CFFFFF770FF4FF00109DFF86880BF
:10333000451A012C05EB01060F4604D8FFF784FF60
:103340000120BDE8F883C8F8109031F8023B3380C3
:10335000FFF75AFF0020C8F8100033883A889BB264
:103360009A420DD040F25D22064B1A60074B1E6058
:10337000074B1C60074B1F60FFF766FFBDE8F88333
:10338000023CD6E700250020FFFF0108F4240020BE
:10339000FC240020F824002000200240084908B541
:1033A0000B7828B153B9FFF739FF01230B7008BD23
:1033B00023B1BDE808400870FFF746BF08BD00BF55
:1033C0000425002038B500F059F94FF47A730C4900
:1033D0000C4A0C6A116803FB04F38B420A49D1E9D9
:1033E000004504D2003445F10105C1E90045E41867
:1033F00045F10005136000F04BF92046294638BD21
:10340000B4240020082500201025002008B5FFF76F
:10341000D9FF4FF47A720023FCF7BAFE08BD00BF53
:1034200010B5094C0439013AD2B2FF2A00D110BDBF
:1034300053089800043054F8233000599BB243EAF3
:10344000004341F8043FEEE7046C004030B5074804
:10345000013AD2B2FF2A00D130BD0D88540840F89D
:103460002450A3004C8804331C50F1E7046C004046
:1034700007B5012201A90020FFF7D2FF019803B090
:103480005DF804FB13B50446FFF7F2FFA04206D037
:1034900002A941F8044D01220020FFF7D7FF02B036
:1034A00010BD00007047000045F25552064B1A60EF
:1034B00002225A6040F6FF729A604CF6CC421A60C3
:1034C0000122024B1A70704700300040192500207D
:1034D000034B1B781BB14AF6AA22024B1A607047B5
:1034E0001925002000300040034B1B689B0042BFA1
:1034F0000122024B1A707047241002401825002048
:103500004FF08072014B1A60704700BF24100240D8
:10351000014B1878704700BF18250020EFF309838E
:10352000203383F30988002383F311887047000058
:1035300010B5202383F311880D4B5B6813F40063EF
:1035400012D0EFF309844FF0807344F8043CA4F1E7
:10355000200383F30988FFF773FD18B1054B44F886
:10356000083C10BD044BFAE783F3118810BD00BF7F
:1035700000ED00E0A1050008A40500087047000068
:10358000FEE70000084A094B09498B4204D3002199
:10359000084A934205D3704752F8040F43F8040BCE
:1035A000F3E743F8041BF4E764410008D425002046
:1035B000D4250020D4250020FEE7000010B5174CCC
:1035C000FFF7B0FCFFF7DCFD802215492046FFF72E
:1035D00061FD012344F8180C0374124B124AD96898
:1035E00021F4E0610904090C0A431049DA60CA6851
:1035F00042F08072CA600E490A6842F001020A6015
:103600001022DA77202283F82220002383F3118806
:1036100062B6BDE810400748FFF75EBDDC2400201D
:103620004840000800ED00E00003FA05F0ED00E07E
:10363000001000E050400008F8B50F4C226A01323B
:103640002262224652F8141F9142154606D02026C7
:103650008B68013B8B6063699A6802B1F8BD196899
:10366000DF68DA604D60616182F311881869B847DC
:1036700086F31188EFE700BFB4240020EFF3118038
:1036800020B9EFF30583202282F3118870470000F0
:1036900010B558B9EFF30584C4F3080414B180F3EE
:1036A000118810BDFFF7ECFC84F3118810BD0000F9
:1036B00000F030B808B500F063F9FFF77FFFBDE810
:1036C0000840FFF711BF0000704700004FF0FF31C6
:1036D0000E4B1A6919611A6900221A611869D868B3
:1036E000D960D968DA60DA68DA6942F08052DA6162
:1036F000DA69DA6942F00062DA61054ADB69136867
:1037000043F48073136000F01BB900BF0010024047
:1037100000700040194B1A6842F001021A601A68E2
:103720009007FCD51A6802F0F9021A6000225A606C
:103730005A6812F00C0FFBD11A6842F480321A60FA
:103740001A689103FCD55A6842F4E8125A601A6864
:1037500042F080721A601A689201FCD51221084A60
:103760005A60084A11605A6842F002025A605A6868
:1037700002F00C02082AFAD1704700BF0010024084
:1037800000641D0000200240084A08B55369116812
:103790000B4003F00103536123B1054A13680BB1D9
:1037A00050689847BDE80840FFF7C2BE00040140DA
:1037B000E4220020084A08B5536911680B4003F061
:1037C0000203536123B1054A93680BB1D06898474F
:1037D000BDE80840FFF7ACBE00040140E422002031
:1037E000084A08B5536911680B4003F0040353619C
:1037F00023B1054A13690BB150699847BDE80840E9
:10380000FFF796BE00040140E4220020084A08B5F4
:10381000536911680B4003F00803536123B1054A53
:1038200093690BB1D0699847BDE80840FFF780BEA7
:1038300000040140E4220020084A08B553691168D9
:103840000B4003F01003536123B1054A136A0BB117
:10385000506A9847BDE80840FFF76ABE000401407F
:10386000E4220020174B10B55C691A68144004F478
:1038700078725A61A30604D5134A936A0BB1D06AD1
:103880009847600604D5104A136B0BB1506B9847EC
:10389000210604D50C4A936B0BB1D06B9847E20517
:1038A00004D5094A136C0BB1506C9847A30504D595
:1038B000054A936C0BB1D06C9847BDE81040FFF7F8
:1038C00037BE00BF00040140E42200201A4B10B5AF
:1038D0005C691A68144004F47C425A61620504D59C
:1038E000164A136D0BB1506D9847230504D5134A42
:1038F000936D0BB1D06D9847E00404D50F4A136E59
:103900000BB1506E9847A10404D50C4A936E0BB1CD
:10391000D06E9847620404D5084A136F0BB1506FFC
:103920009847230404D5054A936F0BB1D06F98478D
:10393000BDE81040FFF7FCBD00040140E422002078
:10394000062108B50846FFF791F806210720FFF782
:103950008DF806210820FFF789F806210920FFF7D6
:1039600085F806210A20FFF781F806211720FFF7C6
:103970007DF8BDE8084006212820FFF777B8000051
:1039800008B5FFF7A3FE0648FEF75EFFFFF78CF8C9
:10399000FFF78EFAFFF798FEBDE8084000F002B886
:1039A0007040000800F00EB808B5202383F311889A
:1039B000FFF742FE002383F31188BDE80840FFF7BC
:1039C000B7BD0000054B064A08215A6000229A60E4
:1039D00007220B201A60FFF75FB800BF10E000E07D
:1039E0003F1901001FB51C46094B05461B68D868E6
:1039F00052B1084B8DE80A0002922B462246064936
:103A0000FDF7B6FC00F042F8044B1A46F2E700BF9F
:103A100014110020AC400008B94000089F3B00088A
:103A200010B501390244904201D1002010BD10F8B8
:103A3000013B11F8014FA342F5D0181B10BD000047
:103A40002DE9F8430746884691461E468BB10D4640
:103A5000A8EB0500B54207EB000402D20020BDE848
:103A6000F883324649462046FFF7DAFF18B1013D98
:103A7000EEE7BDE8F8832046BDE8F883034611F879
:103A8000012B03F8012B002AF9D1704708B5062055
:103A900000F02CF80120FFF7AFFB00001F2938B51C
:103AA00004460D4604D9162303604FF0FF3038BD9D
:103AB000426C12B152F821304BB9204600F030F878
:103AC0002A4601462046BDE8384000F017B8012BD1
:103AD0000AD0591C03D116230360012038BD0024ED
:103AE000284642F825409847002038BD024B014641
:103AF0001868FFF7D3BF00BF1411002038B50023AA
:103B0000064C0546084611462360FFF779FB431C27
:103B100002D1236803B12B6038BD00BFD02500203F
:103B2000FFF768BB40A2E4F1646891064E6F206124
:103B30007070207369670A00426164206677206CA8
:103B4000656E6774682025750A0042616420626FA3
:103B50006172645F69642025752073686F756C6499
:103B60002062652025750A00426164206170702022
:103B7000435243203078253038783A307825303831
:103B800078203078253038783A3078253038780AFF
:103B900000476F6F64206669726D776172650A0015
:103BA00072656365697665645F756E697175655F79
:103BB00069645F6C656E203C2055415643414E5F01
:103BC00050524F544F434F4C5F44594E414D49431F
:103BD0005F4E4F44455F49445F414C4C4F43415415
:103BE000494F4E5F554E495155455F49445F4D41E0
:103BF000585F4C454E475448002E2E2F2E2E2F54E2
:103C00006F6F6C732F41505F426F6F746C6F6164A4
:103C100065722F63616E2E63707000616C6C6F63F0
:103C2000617465645F6E6F64655F6964203C3D200C
:103C3000313237006F72672E6172647570696C6F14
:103C4000742E61705F7065726970685F72616E6713
:103C50006566696E64657200766F69642068616E7E
:103C6000646C655F616C6C6F636174696F6E5F72C9
:103C70006573706F6E73652843616E617264496E1F
:103C80007374616E63652A2C2043616E61726452A5
:103C9000785472616E736665722A290063616E6181
:103CA0007264496E6974000063616E617264536589
:103CB000744C6F63616C4E6F646549440000000092
:103CC00063616E61726448616E646C6552784672BD
:103CD000616D650063616E6172644465636F646504
:103CE0005363616C6172000063616E617264456E62
:103CF000636F64655363616C61720000696E637227
:103D0000656D656E745472616E73666572494400C8
:103D1000656E717565756554784672616D65730081
:103D2000707573685478517565756500707265704B
:103D3000617265466F724E6578745472616E736617
:103D400065720000636F70794269744172726179C3
:103D5000000000006465736361747465725472617D
:103D60006E736665725061796C6F6164000000006B
:103D700066726565426C6F636B0000006269745F18
:103D80006C656E677468203E20300072656D6169F5
:103D90006E696E675F62697473203E203000696EE1
:103DA0007075745F6269745F6F6666736574203ED8
:103DB0003D20626C6F636B5F6269745F6F666673F0
:103DC000657400626C6F636B5F656E645F626974DB
:103DD0005F6F6666736574203E20626C6F636B5F15
:103DE0006269745F6F66667365740072656D6169A0
:103DF0006E696E675F6269745F6C656E6774682078
:103E00003C3D2072656D61696E696E675F626974C1
:103E10007300696E7075745F6269745F6F66667354
:103E20006574203C3D207472616E736665722D3E30
:103E30007061796C6F61645F6C656E202A20380058
:103E40006F75747075745F6269745F6F66667365B1
:103E500074203C3D2036340072656D61696E696E78
:103E6000675F6269745F6C656E677468203D3D20B2
:103E7000300028726573756C74203E20302920262E
:103E8000262028726573756C74203C3D20363429D9
:103E90002026262028726573756C74203C3D2062B4
:103EA00069745F6C656E677468290000646573747B
:103EB000696E6174696F6E20213D202828766F69D4
:103EC00064202A2930290076616C756520213D2007
:103ED0002828766F6964202A293029006F66667366
:103EE00065745F77697468696E5F626C6F636B207D
:103EF0003C2028333255202D205F5F6275696C7439
:103F0000696E5F6F66667365746F66202843616EC5
:103F1000617264427566666572426C6F636B2C20D9
:103F200064617461292900006F75745F696E732084
:103F3000213D202828766F6964202A293029000035
:103F40007372635F6C656E203E2030550000000088
:103F50002863616E5F6964202620307831464646CA
:103F6000464646465529203D3D2063616E5F6964A3
:103F700000000000616C6C6F6361746F722D3E73A2
:103F80007461746973746963732E63757272656E9C
:103F9000745F75736167655F626C6F636B73203EFE
:103FA000203000007472616E736665725F69642010
:103FB000213D202828766F6964202A2930290000B5
:103FC00073746174652D3E6275666665725F626CBE
:103FD0006F636B73203D3D202828766F6964202A2B
:103FE000293029002E2E2F2E2E2F6D6F64756C65B3
:103FF000732F6C696263616E6172642F63616E61BD
:1040000072642E63006974656D2D3E6672616D6524
:104010002E646174615F6C656E203E20300000008C
:1040200000000000792E0008652E0008A12E00086F
:104030008D2E0008992E0008852E0008712E00088C
:104040005D2E0008AD2E00086D61696E0000000055
:104050006840000820250020D02500200100000035
:10406000B93500080000000069646C6500000000BC
:104070000C1E0000887B8188B857898801000000E9
:1040800082888884888888880000000088888888DA
:1040900088888888000000008888888888888888C0
:1040A0000000000088888888888888882C206675A9
:1040B0006E6374696F6E3A20006173736572746920
:1040C0006F6E2022257322206661696C65643A2038
:1040D00066696C6520222573222C206C696E652030
:1040E0002564257325730A00D8C0FF7F01000000F6
:1040F000FFFFFFFF6400000000000000FE2A010037
:10410000D204000018110020000000000000000090
:10411000000000000000000000000000000000009F
:10412000000000000000000000000000000000008F
:10413000000000000000000000000000000000007F
:10414000000000000000000000000000000000006F
:10415000000000000000000000000000000000005F
:08416000000000000000000057
:00000001FF
